:100000000C94DC020C94F9020C9414030C94F90285
:100010000C94F9020C94F9020C94F9020C94F90274
:100020000C94F9020C94F9020C943B220C94F90202
:100030000C94F9020C94F9020C94F9020C94F90254
:100040000C94F9020C94F9020C94F9020C94F90244
:100050000C94F902B706B706E306E3064B077608E9
:1000600076087608690702081308130829001E009D
:100070001F0020002100220023002400250026006C
:1000800027002D002E0035002B0014001A00080058
:10009000150017001C0018000C00120013002F00A0
:1000A00030002A00390004001600070009000A0089
:1000B0000B000D000E000F0033003400000028007C
:1000C000E10000001D001B000600190005001100E2
:1000D0001000360037003800E5005200E000E30071
:1000E000E200000000002C0000000151E4000000CC
:1000F0000000500051004F0002514E004B00000024
:1001000000000000000000000000000000000000EF
:1001100000000000000000000000000000000000DF
:1001200000000000000000000000000000004C0083
:1001300035003A003B003C003D003E003F004000DF
:10014000410042004300440045003100C05CC15CF6
:10015000BF5CBE5C005C0100010001000100010009
:100160004600010001000100C35CC45CC65CC85CC1
:10017000CA5CCC5C0100010001000100010001002B
:100180000000010001000000C55CC75CC95CCB5CDD
:10019000CD5C01000100010001000100010001002F
:1001A000010001000100000000000100000001004A
:1001B00001000000000001000100010001004D00ED
:1001C0004A000000000000000000000000000000E5
:1001D000000000000000000000000000000000001F
:1001E000000000000000000000000000000000000F
:1001F00000004C0035000100010001000100010079
:1002000001000100010001000100AA00A900010095
:1002100001000100010001000100010001000100D6
:100220000100010046000100010001000100010081
:1002300001000100010001000100010001000100B6
:1002400001000100000001000100000001000100A8
:100250000100010001000100010001000100010096
:100260000100AE00010001000100000000000100DB
:1002700000000100010000000000AC00AD00AB0078
:10028000010001000100000000000000000000006B
:10029000000000000000000000000000000000005E
:1002A000000000000000000000000000000000004E
:1002B000000000000000010000047F3F1F643214B2
:1002C000643214783C1E1E140A0522232526282990
:1002D0002A2C2D2F3032333536383A3B3D3E4042C2
:1002E000434547494A4C4E5051535557595A5C5E05
:1002F0006062646668696B6D6F71737577797B7D19
:100300007F81838587898A8C8E90929496989A9C17
:100310009E9FA1A3A5A7A8AAACAEAFB1B3B4B6B82F
:10032000B9BBBCBEBFC1C2C3C5C6C7C9CACBCCCD91
:10033000CED0D1D2D2D3D4D5D6D7D7D8D9D9DADA6C
:10034000DBDBDBDCDCDCDCDCDDDDDDDDDCDCDCDCEC
:10035000DCDBDBDBDADAD9D9D8D7D7D6D5D4D3D220
:10036000D2D1D0CECDCCCBCAC9C7C6C5C3C2C1BFFE
:10037000BEBCBBB9B8B6B4B3B1AFAEACAAA8A7A562
:10038000A3A19F9E9C9A98969492908E8C8A89871E
:100390008583817F7D7B79777573716F6D6B6968FC
:1003A000666462605E5C5A5957555351504E4C4AD0
:1003B0004947454342403E3D3B3A3836353332307B
:1003C0002F2D2C2A292826252322FFAA7F554000DD
:1003D0000101010101010101010202020202020206
:1003E00002020303030303030303040404040404D9
:1003F000040505050505060606060607070707079F
:1004000008080808090909090A0A0A0B0B0B0C0C51
:100410000C0D0D0D0E0E0E0F0F0F101011111112ED
:100420001213131414151516161717181819191A6C
:100430001A1B1B1C1D1D1E1E1F20202122222324CF
:1004400024252626272829292A2B2C2D2D2E2F300E
:10045000313232333435363738393A3B3C3D3E3F22
:10046000404142434445464748494A4C4D4E4F500F
:10047000515354555658595A5B5D5E5F61626465CD
:100480006668696B6C6D6F7072737577787A7B7D57
:100490007E8082838587888A8C8E8F9193959698AB
:1004A0009A9C9EA0A2A3A5A7A9ABADAFB1B3B5B7C7
:1004B000BABCBEC0C2C4C6C9CBCDCFD1D4D6D8DB9E
:1004C000DDDFE2E4E7E9EBEEF0F3F5F8FAFDFF0932
:1004D000023B00020100A0FA09040000010301012F
:1004E00000092101010001224000070581030800E5
:1004F00001090401000103000000092101010001BC
:1005000022320007058303080001120110010000D8
:10051000000847540091010001020001100354003B
:10052000470052002D003900310030000000120356
:100530005100750061006400630075006200650091
:1005400000000403090405010980A10185031901C4
:100550002AB700150126B700950175108100C00566
:100560000C0901A101850419012AA002150126A088
:1005700002950175108100C005010906A10105075A
:1005800019E029E7150025019508750181029501FB
:10059000750881030507190029FF150026FF00953E
:1005A0000675088100050819012905950575019151
:1005B00002950175039103C011241FBECFE5D8E059
:1005C000DEBFCDBF11E0A0E6B0E0E4E0FDE402C094
:1005D00005900D92A232B107D9F723E0A2E2B1E073
:1005E00001C01D92A633B207E1F70E944F140C948C
:1005F00080260C940000A82FB92F80E090E041E005
:1006000050EA609530E009C02D9182279795879533
:1006100010F084279527305EC8F36F5FA8F3089524
:10062000EADF8D939D930895CF93CFB7CF93C39572
:10063000839BE9F7839B0EC0839B0CC0839B0AC0FE
:10064000839B08C0839B06C0C0910D03C395C093D4
:100650000D03A6C0DF93C0910C03DD27CC5EDC4FF9
:10066000839B02C0DF91E6CF2F930F931F9300B3BC
:100670002FEF03FB20F94F933F9310B34FEF012768
:1006800003FB21F93BE031C04E7F012F10B3216005
:1006900028C0102F4D7F2260000000B329C04B7F7F
:1006A0002460012F000010B32BC010B3477F2860D7
:1006B0002AC04F7E00B320612CC04F7D10B3206252
:1006C0002FC04F7B00B3206432C0422700B3499350
:1006D0004FEF0000102713FB20F910B31C70C9F175
:1006E000297F91F2012703FB21F900B3237F89F2CF
:1006F000315058F1102713FB22F910B3277E79F2FD
:10070000012703FB23F92F7C81F200B3102713FB91
:1007100024F92F7971F200C010B3012703FB25F9EA
:100720002F7359F200C000B3102713FB26F92230B3
:1007300040F200C010B3012703FB27F9243028F64C
:100740004F77206810B30000F9CF10E81ABF0027D8
:100750001CC03B503195C31BD04010E81ABF088124
:10076000033C11F10B3401F1209109031981110FA0
:100770001213EDCF4A81441F093669F10D3211F091
:10078000013E29F74F7009F0042F009312033F91A7
:100790004F911F910F912F91DF91CAB7C7FD47CF9E
:1007A000CF91CFBFCF91189520911203222379F3D7
:1007B00010911003112309F044C034300AF443C0EF
:1007C0003093100320930B0310910C033BE0311B7B
:1007D00030930C0338C000911003013094F50AE502
:1007E0004F7049F43091840034FD2FC00093840091
:1007F000C6EED2E02EC0433059F0443091F0309133
:10080000F10234FD22C00093F102C2EFD2E021C018
:1008100030912A0334FD19C000932A03CBE2D3E0C0
:1008200018C03091FD0234FD10C00093FD02CEEFE0
:10083000D2E00FC02795A8F45150A9F4220F000070
:10084000F9CF4AE503C042ED01C0432FC4E1D0E037
:1008500032E011B31C60939A11BB02B320E41CE098
:100860005F93012756E002BB279520F4515021F4F5
:10087000220FF9CF012756E000003B5A02BBD0F20D
:10088000279528F4515029F4220F0000F9CF0127B1
:1008900056E0279502BB20F4515021F4220FF9CFE6
:1008A000012756E02991332302BB21F6037F1091E3
:1008B0001103110FC651D04002BB11F01093090370
:1008C00010E81ABF086011B3137F402F437F5F9178
:1008D00000C000C002BB11BB42BB59CF81E00895EC
:1008E00081E008950C94700408950C9474041F938F
:1008F000CF93DF9300D000D01F92CDB7DEB74983EE
:100900005A836B833091250189819A81311114C0FA
:10091000662359F0222349F00E94AF0A182F682F4E
:1009200089819A810E94580A03C00E94830A182F65
:1009300069817A81812F04C00E94AF0A69817A811E
:100940000F900F900F900F900F90DF91CF911F910C
:100950000C94D711FC01262F408151816281738153
:1009600084810C94770481E00895CF93DF93EC01A8
:1009700060E00E94AA04BE01DF91CF910C9475043F
:100980000C9406130C94021308950E9402090E940D
:10099000C4042FEB87E299E0215080409040E1F7BA
:1009A00000C000000C9461220F931F93CF93DF933C
:1009B0008C0161E00E94AA04EC01B8010E9472045B
:1009C000882309F44BC0B801CE010E944A1C882339
:1009D00009F444C0B801CE010E941D208823F1F122
:1009E000B801CE010E94491D8823C1F1B801CE0192
:1009F0000E94791F882391F1B801CE010E948E1ABE
:100A0000882361F1F8018281882309F1CB358DE5D6
:100A1000D807C1F050F4C115FCE5DF0781F0CF3DE8
:100A2000DC45A9F40E94E00F19C0CC35EDE5DE07E6
:100A300061F0CD35DD4559F40E94290F08C00E94B0
:100A4000C5040CC00E94320F02C00E94350FC801BD
:100A5000DF91CF911F910F910C946E0480E0DF9194
:100A6000CF911F910F9108950E94E52180E00E948F
:100A70007F1C0C946D050E946E1B0E9470050C94E7
:100A8000EB2108950C94410581E00895CF93C82F80
:100A90000E944405882379F0C0FF02C0909A01C0EB
:100AA0009098C1FF02C0919A01C09198C2FF02C004
:100AB000969A01C09698CF910895889A9098899AAD
:100AC00091988E9A96980895CF93C82F0E944205C8
:100AD0008C2F0E944605CF91089580E00C94640508
:100AE0000E9452210C9464050E945221909124018D
:100AF000891721F0809324010C9464050895CF9305
:100B0000DF93CDB7DEB72B970FB6F894DEBF0FBEDD
:100B1000CDBF4F83588769877A878B8761110E9481
:100B2000750E9E012F5F3F4F86E0F90111928A9565
:100B3000E9F785E0FE013796D90101900D928A957B
:100B4000E1F789819A814C815D81452B31F09F3F8E
:100B500031F491E08F3F19F403C091E001C090E0BF
:100B600090FF09C049815A816B817C818D819E8172
:100B70000E94960D05C0C9010E94B3048111F2CFF5
:100B80002B960FB6F894DEBF0FBECDBFDF91CF918D
:100B90000895FC01808191810E94F10A0895CF930C
:100BA000882309F44DC0C82F8CEF8C0F813AF8F4DC
:100BB0008C2F0E943D1F811143C06C2F80916200D9
:100BC000909163000E94A121882349F06C2F8091AD
:100BD0006200909163000E94D9210E94970E6C2FB1
:100BE00080916200909163000E94D7210CC080E246
:100BF0008C0F883058F4C77081E001C0880FCA9507
:100C0000EAF70E94580ECF910C94970EEBE5EC0F8B
:100C1000E33040F4F0E0ED54FF4F808190E0CF915D
:100C20000C946921C85AC73158F4EC2FF0E0EE0F4C
:100C3000FF1FEB57FF4F80819181CF910C947F2153
:100C4000CF910895882349F1682F8CEF860F813A60
:100C500038F480916200909163000E94D9210CC009
:100C600080E2860F883050F4677081E001C0880F01
:100C70006A95EAF70E945E0E0C94970E8BE5860F3C
:100C8000833020F480E090E00C946921685A673149
:100C900020F480E090E00C947F2108951F93CF937F
:100CA000DF93182FEB010E94CF05209741F087EBCF
:100CB0009BE00197F1F700C000002197F6CF812F4C
:100CC000DF91CF911F910C942206893319F060E0D7
:100CD00070E002C060E570E00C944E06882321F0BD
:100CE0000E94580E0C94970E0895882321F00E94BC
:100CF0005E0E0C94970E0895CF92DF92EF92FF92C2
:100D00000F931F93CF93DF937C01D62FC72FFC0146
:100D10001281058102950F700E944E0E8823B9F052
:100D20001123A9F08C2F807F803421F080E28D0F79
:100D3000883068F08091860282FD09C082E00E94BE
:100D4000F70E0E944E0E91E0D82ED92601C0D12C6C
:100D5000CC2EC2948FE0C8228C2D90E08C3091056F
:100D600008F0C4C1FC01E65DFF4F0C94CF258C2F29
:100D7000807FCF70882311F0C295C07F112399F036
:100D8000CC2309F49FC180E28D0F883010F0D1117F
:100D900004C08C2F0E94580E03C08C2F0E94680E36
:100DA0000E94970E8FC18D2F0E942206CC2309F43A
:100DB0009DC180E28D0F883038F1DD2329F18C2F21
:100DC0000E946E0E24C08C2F807FCF70803211F075
:100DD000C295C07FDD2319F0D130A1F13DC08091D3
:100DE000860282FF17C0112349F0CC2329F08C2FF3
:100DF0000E94580E0E94970E80E065C180E00E941C
:100E00002206CC2309F472C18C2F0E945E0E0E9430
:100E1000970E6CC1112371F0002341F0013031F4C1
:100E20000E94780E8C2B0E94800E60C10E94780E6A
:100E30008C2B1DC0002319F0013009F457C10E940A
:100E40008D0E25C0112321F0063008F04FC10EC0D1
:100E5000053008F04BC11BC0112361F0002331F0B5
:100E6000F701858180FF2EC18F7085838C2F0E94B2
:100E70006E063CC1002359F0D93309F034C1FFEFAD
:100E80000DEE12E0F15000401040E1F72AC18C2F26
:100E90000E9475062BC18C2F86958695837019F05C
:100EA000813061F023C1112321F08D2F9C2F93708D
:100EB00002C080E090E00E94692120C1112321F04E
:100EC0008D2F9C2F937002C080E090E00E947F21C4
:100ED00015C18C2F837009F047C011110BC12D2F44
:100EE000229526952770220F220F6D2F6F70862F67
:100EF00090E0A0E0B0E0022E04C0880F991FAA1F66
:100F0000BB1F0A94D2F7D4FF10C04FE050E060E05E
:100F100070E004C0440F551F661F771F2A95D2F753
:100F2000409550956095709503C040E050E0BA013F
:100F3000C695C695C3708A019B01082B192B2A2BD5
:100F40003B2BC901B801C23049F058F4C13019F047
:100F50000E946E09CFC00E945C09CCC00E9480092B
:100F6000C9C00E945A09C6C0112319F08C2F817084
:100F700001C08695882309F4BDC02D2F22952695A2
:100F80002770220F220F6D2F6F70862F90E0A0E048
:100F9000B0E0022E04C0880F991FAA1FBB1F0A943D
:100FA000D2F7D4FF10C04FE050E060E070E004C022
:100FB000440F551F661F771F2A95D2F7409550950D
:100FC0006095709503C040E050E0BA01C695C695A3
:100FD000C3708A019B01082B192B2A2B3B2BC901BB
:100FE000B801C23049F058F4C13019F00E94330AF8
:100FF00081C00E94210A7EC00E94450A7BC00E94D7
:10100000940978C0CF70112339F08C2F0E94BA094F
:101010008D2F0E946E066EC08D2F0E9475068C2F3C
:101020000E94DB0967C0D23F21F128F4D03F41F094
:10103000D13FC1F043C0D33F19F1D43F79F03EC056
:10104000112341F0053008F051C08C2F8F710E94A0
:10105000000A4CC0063008F049C0F7CF80918602E4
:1010600082FF18C0112339F08C2F8F710E94BA09AA
:101070003DC01123C9F38C2F8F710E94DB0936C04C
:10108000112329F08C2F8F710E94A5092FC00E9477
:10109000A0092CC0112349F0CF718C2F0E94BA09EE
:1010A00063E08C2F0E94DC0E21C081E00E94F70ECD
:1010B0000230E0F082E00E94F70E18C0112331F0F8
:1010C000002391F28D2F0E94CF0510C0002399F2CA
:1010D000D93349F41FEF2DEE32E01150204030405B
:1010E000E1F700C000008D2F0E94220688EF8C0DD2
:1010F000843020F40E9452210E946405DD20C9F052
:101100000E944A0E80FD15C0F70112820E94440E13
:101110000E94BA09C7010E94BA080E94440EDF91DA
:10112000CF911F910F91FF90EF90DF90CF900C9493
:10113000DB09DF91CF911F910F91FF90EF90DF902E
:10114000CF9008950F931F93CF93DF93EC016881A5
:1011500079818A810E94FC0A8C010E94570A0E94B0
:101160004809B801CE010E947C06DF91CF911F9102
:101170000F910895CF93DF93EC01988189812B81A2
:101180003C81232B31F08F3F31F481E09F3F19F4F4
:1011900003C081E001C080E080FD1DC0CE010E943F
:1011A000D404811110C00E944E0E8823A1F08A81C0
:1011B000882389F08091860282FD0DC082E0DF9154
:1011C000CF910C94F70ECE010E94A208CE01DF91C0
:1011D000CF910C94B504DF91CF91089580E090E019
:1011E0000E94692180E090E00E947F210E94750E9C
:1011F0000C94970E80916200909163000E94DB2115
:101200000C94EE080E94650E0C94FA0892959F705B
:10121000963079F010F4925001C09A50923068F4F0
:10122000803F69F018F4883E40F409C0843F29F4F7
:1012300006C0883E20F0813F11F080E0089581E0F3
:101240000895FC01808191810E94F10A0E940609A3
:101250000895CF93DF9300D000D01F92CDB7DEB7B3
:101260000F900F900F900F900F90DF91CF910895F6
:10127000CF93DF9300D000D000D0CDB7DEB7269655
:101280000FB6F894DEBF0FBECDBFDF91CF910895AA
:10129000089508950C9449090C944A090E944C0938
:1012A00060936B0170936C0180936D0190936E015C
:1012B0000C94EE080C944E090F931F9300916B0150
:1012C00010916C0120916D0130916E01602B712B9A
:1012D000822B932B1F910F910C944E090F931F9308
:1012E00000916B0110916C0120916D0130916E01A4
:1012F00060237123822393231F910F910C944E0935
:101300000F931F9300916B0110916C0120916D015F
:1013100030916E0160277127822793271F910F91CB
:101320000C944E090C9449090E949209609367013C
:10133000709368018093690190936A010C94EE08A0
:1013400060E070E0CB010C9494090F931F9341E08F
:1013500050E060E070E08A019B0104C0000F111FA3
:10136000221F331F8A95D2F7C901B8011F910F912F
:101370000C9494090F931F9341E050E060E070E0FB
:1013800004C0440F551F661F771F8A95D2F78091BE
:10139000670190916801A0916901B0916A018A0189
:1013A0009B01082B192B2A2B3B2BC901B8011F913C
:1013B0000F910C9494090F931F9341E050E060E06B
:1013C00070E004C0440F551F661F771F8A95D2F73F
:1013D0004095509560957095809167019091680156
:1013E000A0916901B0916A018A019B010823192328
:1013F0002A233B23C901B8011F910F910C94940932
:101400000F931F9341E050E060E070E004C0440F90
:10141000551F661F771F8A95D2F7809167019091BB
:101420006801A0916901B0916A018A019B010827B6
:1014300019272A273B27C901B8011F910F910C9446
:1014400094090F931F9300916701109168012091F7
:10145000690130916A01602B712B822B932B1F91B4
:101460000F910C9494090F931F93009167011091B1
:1014700068012091690130916A0160237123822300
:1014800093231F910F910C9494090F931F93009134
:101490006701109168012091690130916A0160270C
:1014A0007127822793271F910F910C949409089517
:1014B0002EE0929F800D1124E82FE695E695E695A3
:1014C000877051E001C0550F8A95EAF785E0E89FE3
:1014D000F0011124EA5DFE4F20E030E070E0408131
:1014E000CB01022E02C0969587950A94E2F781708F
:1014F000819584278523842781932F5F3F4F253053
:10150000310569F708952EE0929F800D1124682F10
:10151000669566956695982F977085E0689FB001EF
:10152000112440E050E080E0FB01E40FF51FEA5D8C
:10153000FE4F208130E0092E02C0369527950A948F
:10154000E2F721703327042E01C0220F0A94EAF734
:10155000822B4F5F5F4F4530510531F70895BF92A1
:10156000CF92DF92EF92FF920F931F93CF93DF936F
:101570008C01C0906701D0906801E0906901F09003
:101580006A0180916B0190916C01A0916D01B09105
:101590006E01C82AD92AEA2AFB2ACFE1D0E0D70176
:1015A000C6010C2E04C0B695A795979587950A9409
:1015B000D2F780FD04C0219790F7B12C07C0BC2E54
:1015C000B8018C2F0E94EA110197A9F38B2DDF91AE
:1015D000CF911F910F91FF90EF90DF90CF90BF9030
:1015E0000895CF93DF93EC010E94AF0ABE010E94E1
:1015F000EA11DF91CF9108951F93CF93DF93EB0111
:1016000090912501992321F0CB010E94F10A13C08A
:10161000882349F0CB010E94AF0A182F682FCE0112
:101620000E94580A04C0CB010E94830A182FBE01F1
:10163000812F0E94EA11DF91CF911F9108951F938E
:10164000CF93DF93C0916F0116E080917001C817AE
:1016500099F0D0E01C9FF0011D9FF00D1124EF5870
:10166000FE4F4081518162817381848195810E9406
:1016700038092196C770E9CFDF91CF911F91089566
:101680004091A1015091A2016091A3017091A40128
:101690008091A5019091A6010C943809EF92FF92D8
:1016A0000F931F93CF93DF938091A60182958F7044
:1016B00009F065C08091A301882309F460C080917E
:1016C0006F01F09070011091A1010091A201609151
:1016D000A4017091A50191E01F3F09F090E0C09135
:1016E0006000D0916100292F96E0E92E8F1509F452
:1016F00046C06115710521F00F3F21F030E003C0B5
:1017000031E001C0322F90E030FD36C0E89EF0019C
:10171000E99EF00D1124DF01AF58BE4F11963C91A8
:101720001197301329C03C91311326C012963C9179
:101730001297311121C013964D915C911497461B5D
:10174000570B4C175D07C0F48091A6018F70806124
:101750008093A601EA58FE4F80818F70806180835C
:1017600081EA91E00E94BA08DF91CF911F910F9119
:10177000FF90EF900C941F0B01968770B7CFDF910D
:10178000CF911F910F91FF90EF9008959F92AF928C
:10179000BF92CF92DF92EF92FF920F931F93CF935E
:1017A000DF93CDB7DEB761970FB6F894DEBF0FBEFB
:1017B000CDBF8C0185E0F801DE011D9601900D92F0
:1017C0008A95E1F7D8011296EC909091A101E091F1
:1017D000A2012091A4013091A5012115310531F01C
:1017E000EF3F31F481E09F3F19F403C081E001C075
:1017F00080E0B82FB1709B2E80FD47C1D8014C917D
:1018000011965C9111971396AD90BC90149781EA54
:10181000C82E81E0D82EF090A301B501621B730B96
:101820002091600030916100FF2009F4D9C08091BF
:10183000A6016217730708F095C0282F207F09F0D2
:1018400052C05E1313C0491311C0FE2CE1100EC02C
:101850008F7080618093A6010E94400BC6010E9498
:10186000BA088091A601F80185834DC1AB2831F0FB
:101870005F3F31F481E04F3F19F403C081E001C0C4
:1018800080E080FD03C081E08E2502C080E090E012
:10189000F82FF170FF2E80FF1CC080916F01209106
:1018A000700136E0821709F40BC190E0389FF00117
:1018B000399FF00D1124EF58FE4F6181561306C079
:1018C0006081461303C06281E61203C001968770EF
:1018D000E9CFFE2CEE2009F416C18091A6018160AB
:1018E0008093A60154C05E1306C0491304C0E110E2
:1018F00002C0F80199C0C8010E942109882361F142
:10190000EE2051F12091A601822F82958F7090E0F8
:10191000029774F08091A1019091A20198878F8322
:101920001986BB86AA862C87CE0107960E94BA0824
:1019300086E0F801A1EAB1E001900D928A95E1F705
:101940000E944E0B0E94400B0AC05E1711F1C801A5
:101950000E94210981112CC0C8010E94BA08FF24ED
:10196000F394D1C0282F207F81F77A2DB98AA88AD5
:101970006E2D89890E94290981EA91E00E94BA08A6
:1019800086E0D6011D928A95E9F70E94400BF12C62
:10199000BAC04913DCCFE110DACFF8018583C80162
:1019A0000E94BA0886E0D6011D928A95E9F7ABC07D
:1019B000EE2091F22091A601822F82958F7090E007
:1019C00002970CF4B5CF8091A1019091A2019A8366
:1019D00089831B82BD82AC822E83CE010196A6CF65
:1019E0006217730708F044C0FE2CEE2009F4B4CF50
:1019F0005E1330C049132EC02091A60120FD21C0E6
:101A0000822F82958F70482F50E041155105C9F003
:101A1000F80125834F30510541F08F5F982F929543
:101A2000907F822F8F70892B8583C8010E94BA080E
:101A300086E0F801A1EAB1E001900D928A95E1F704
:101A40003CC086E0F801A1EAB1E001900D928A95D0
:101A5000E1F759C0C8010E942109811169CF809125
:101A6000A60181608093A601C8010E94BA084BC0FC
:101A70007A2DB98AA88A6E2D89890E94290986E063
:101A8000D6011D928A95E9F718C0EE2009F464CFBB
:101A9000C8010E942109F82E882309F45DCF86E051
:101AA000F801A1EAB1E001900D928A95E1F781EA8F
:101AB00091E00E94C9050E944E0B0E94400B23C07A
:101AC0004D875E878D859E850E94F10A292F22957C
:101AD0002F70223028F49F7039F0811105C00BC09F
:101AE000243028F49F7049F4805E883020F0C801CB
:101AF0000E94BA089F2CF92C06C0D80115969C911B
:101B0000907F91F7F8CF8F2D61960FB6F894DEBFD6
:101B10000FBECDBFDF91CF911F910F91FF90EF903E
:101B2000DF90CF90BF90AF909F9008951F93CF9379
:101B3000DF93CDB7DEB72C970FB6F894DEBF0FBE9C
:101B4000CDBF4F83588769877A878B879C87CE0163
:101B500007960E94C60B8823D1F09F8188852A852D
:101B60003B85232B31F08F3F31F481E09F3F19F407
:101B700003C081E001C080E080FD47C04F815885EF
:101B800069857A858B859C850E9438093EC086E0F0
:101B9000FE013796DE01119601900D928A95E1F7CC
:101BA000FF81E8856A857B856115710531F0EF3F1E
:101BB00031F481E0FF3F19F403C081E001C080E00F
:101BC00080FD23C02091700130E0C901019687702B
:101BD000992740916F0150E084179507F1F1F9833F
:101BE000EA837D836C8396E0929FD001939FB00D32
:101BF0001124AF58BE4FFE01319601900D929A9577
:101C0000E1F7809370010E941F0B16E080916F0135
:101C100090917001891771F1189FC00111248F589C
:101C20009E4F0E94C60B882329F1E0916F011E9FF1
:101C3000F0011124EF58FE4F408151816281738180
:101C4000848195810E94380980916F0190E001960E
:101C50008770992780936F01D9CF0E940209109253
:101C6000700110926F01E1EAF1E086E0DF011D9260
:101C70008A95E9F72C960FB6F894DEBF0FBECDBF5C
:101C8000DF91CF911F9108958091AF018595859542
:101C9000859508958091AF01877008959091AF0167
:101CA000977081E009F480E008958091BA01089569
:101CB0009091BA01892B8093BA01089580959091F3
:101CC000BA0189238093BA0108951092BA01089548
:101CD0009091B901892B8093B901089580959091D5
:101CE000B90189238093B90108951092B90108952B
:101CF0008091B001089508950C947B0E0C947C0E95
:101D00009091860292FD08C09091B001981721F041
:101D10008093B0010C947E0E08958091B0018823C9
:101D200029F01092B00180E00C947E0E0895CF93BC
:101D3000DF93E0916200F09163008091BA018083AB
:101D4000E0916200F091630090818091B901892B4C
:101D500080838091B001882381F0E0916200F0914E
:101D600063009081892B8083809162009091630051
:101D70000E94952181110E948D0EC0916200D09128
:101D8000630048E050E067EA71E0CE010E941F2640
:101D9000892B69F088E0FE01A7EAB1E001900D927D
:101DA0008A95E1F7CE01DF91CF910C945E21DF910E
:101DB000CF9108950C947B0E9091860292FD10C0F5
:101DC00098E0899F90011124262B2093AF010E9457
:101DD000BA098091AF018595859585950C94DA0EA9
:101DE0000C94BA091092AF0180E00C94DA0E2091A5
:101DF000AF01809582238093AF01982F977099F45B
:101E000030E0482F082E000C550B2417350759F0E9
:101E10009091860292FD07C08595859585950E94D3
:101E2000DB090C94F20E08959091860292FB222712
:101E300020F9281769F080FB92F99093860280912F
:101E40008502909186020E945C0F82E00C94F70E4E
:101E500008958091860282FB882780F991E0892786
:101E60000C94140F81E00C94140F80E00C94140F68
:101E700080E090E00E943A2621E0893E9E4F09F0E2
:101E800020E0822F089582E090E00C942C2683E0DD
:101E900090E00C942C26CF9384E090E00E942C26B6
:101EA000C82F82E290E00E942C262C2F30E0A9015E
:101EB000582BCA01CF910895CF93C92F682F84E082
:101EC00090E00E9440266C2F82E290E0CF910C942B
:101ED0004026AB01BC018FE090E00C945126AB0191
:101EE000BC0183E190E00C94512660E070E0CB01EE
:101EF0000C946F0F60E070E0CB010E94690F0C94AE
:101F0000750F69EE7EEF80E090E00E945D2660E054
:101F100082E090E00E94402660E083E090E00E9432
:101F2000402610926B0110926C0110926D0110927C
:101F30006E0160E084E090E00E94402660E082E272
:101F400090E00E94402660E085E090E00E944026FC
:101F500060E086E090E00E9440266FEF87E090E02E
:101F60000E94402640E050E0BA0188E090E00E94E4
:101F7000512660E08DE090E00E94402640E050E075
:101F8000BA0188E190E00E94512660E087E190E08C
:101F90000E94402640E050E0BA018CE190E00E94AF
:101FA000512660E070E080E290E00E945D2640E013
:101FB00050E0BA0188E190E00E9451260C947A0F1B
:101FC0000C94810F682F8EE090E00C9440260E94C4
:101FD00020226093CD017093CE018093CF01909326
:101FE000D0016093C9017093CA018093CB01909393
:101FF000CC01089584B7806884BF84B7806884BFAB
:10200000089581E008950C94011008950C94051032
:102010000C9405100C9408100C9405100C940C10E2
:102020000C9405100E94FA0F86EC92E10E94482160
:102030000E9410100C940E100E9406100C940510B3
:102040000E94C9120E945D050C941F1D0E940D2262
:102050000E94AE130E9420100E946E1B0E94AD19B8
:102060000C940A105F926F927F928F929F92AF9220
:10207000BF92CF92DF92EF92FF920F931F93CF9375
:10208000DF93CDB7DEB72A970FB6F894DEBF0FBE49
:10209000CDBF0E94C313C82E81110E94E70F3BEBF6
:1020A000832E31E0932E00E010E0502E802F0E940E
:1020B000ED125C01F401619071904F016826792660
:1020C00061147104B1F40F5F1F4F0730110569F7F8
:1020D0008FEF89838A831B820E9414228160782F6C
:1020E0009D838C8349815A816B818D810E947F05FC
:1020F0003AC08091D10181FD0E94F612D12CEE24CC
:10210000E394F12CC3018E219F21892B29F10E9498
:1021100003108823A9F0DE825F82AE20BF2081E019
:10212000AB2809F480E088870E9414228160782F10
:102130009A8789874E815F8168858A850E947F059D
:10214000000F111FF801E554FE4F80819181E826B0
:10215000F926F182E08207C0D394EE0CFF1CFEE06A
:10216000DF12D0CFB0CF81E0C11001C080E02A964D
:102170000FB6F894DEBF0FBECDBFDF91CF911F9198
:102180000F91FF90EF90DF90CF90BF90AF909F9016
:102190008F907F906F905F9008950E9432100E9400
:1021A000E0190E941E1D0C947405CF93DF930E94CA
:1021B000EF11EC01811522E59207E8F5811531E573
:1021C000930708F0B6C0883E910528F5803E91053A
:1021D00008F0E9C0883A910570F4853A910508F055
:1021E0007AC08130910509F473C008F4D9C004970E
:1021F00008F0D9C0D5C08F3B910508F0D1C0C85AAE
:10220000D0E0CC0FDD1FCA54DF4F0990D881C02D1C
:10221000CE019464C9C0811540E5940708F069C0F7
:10222000811550E4950708F060C09A9581159F418B
:1022300008F4B9C0B5C0811536E5930728F58115B6
:1022400045E5940708F092C0811554E5950708F01C
:1022500087C0AC0143705527282F26952695C115B8
:10226000D34508F06CC081E090E002C0880F991F50
:102270004A95E2F740E2249F90011124EC01C22B21
:10228000D32BCE019C6890C081152AE5920780F47B
:10229000811539E5930708F072C0811548E5940768
:1022A00008F47EC0D82FCC27CE01806F906A7CC006
:1022B00090568115904208F073C08D2F8F710E9447
:1022C0008312DD27D0628F71AE01582BCA016CC01A
:1022D00081E090E069C0C55AD0E0CC51DF4F8881E1
:1022E000C82FD0E0CE0190645FC0DF70CE01906A4D
:1022F0005BC074E0969587957A95E1F7282F237057
:102300003C2F337081E090E002C0880F991F3A950E
:10231000E2F79C68AC01522B9A019C2F9F70969516
:10232000969550E2959FE0011124C9018C2B9D2BBD
:102330003BC0D82FCC27CE01816F906A35C081E099
:1023400090E002C0880F991F4A95E2F750E2259F5E
:1023500090011124EC01C22BD32BCE019A6824C02A
:10236000D82FCC27CE01846F906A1EC00E948312A2
:102370008F7190E0D82FCC27CE01906215C08F705E
:102380000E94831294E0D695C7959A95E1F7CF7095
:10239000D0E0DC2FCC27D0699E01282BC90104C0D6
:1023A00080E090E001C0CE01DF91CF91089522E658
:1023B000829FC0011124FC012EE0729FE00DF11DEF
:1023C0001124E60FF11DEE0FFF1FE459FF4F859119
:1023D000949108950E94D7110E94D51008958238D3
:1023E000910569F1B0F48133910509F46DC048F4A9
:1023F0008932910509F463C08A32910509F469C0F4
:1024000008958533910509F455C089339105B9F0D4
:102410000895833E910569F138F4803E9105B1F04D
:10242000823E910509F10895863E9105A9F1873E06
:102430009105B9F1843E910509F064C023C0209153
:10244000850220FD4FC021FD4DC008958091850279
:1024500080FD44C08091860280FF44C08091850247
:1024600084FD42C083EE4DC08091850282FF38C05A
:10247000F5CF8091850282FD33C08091860280FD78
:1024800031C0ECCF8091860281FF32C080918502FD
:1024900084FD2AC087EE35C08091850283FF26C067
:1024A000F5CF8091850283FD21C08091860281FD58
:1024B0001FC0ECCF8091850285FD1CC01DC080919E
:1024C000850285FD19C016C08091850286FD16C063
:1024D00017C08091850286FD13C010C089E311C02A
:1024E00082EE0FC080EE0DC080E00BC086EE09C00A
:1024F00084EE07C089E205C085E303C08AE201C01B
:1025000081E390E008959091850292FF0DC0282FFD
:102510002871283019F4877F846006C0282F247121
:10252000243011F48B7F886093FF0DC0282F287111
:10253000283119F4877E846106C0282F2471243144
:1025400011F48B7E88612091860220FF0DC0382F08
:102550003871383019F4877F816006C0382F3171A7
:10256000313011F48E7F886021FF0DC0282F287133
:10257000283119F4877E816106C0282F217121310D
:1025800011F48E7E886194FD877E089580E0089521
:1025900008950E94380F811102C00E94E00F0E942E
:1025A000430F8093D1010E944B0F9093860280933A
:1025B00085020E94C8120E94470F682F70E080E0D9
:1025C00090E00E945A0960916701709168018091C2
:1025D000690190916A010C949209E82FF0E0EE0FE6
:1025E000FF1FEB56FD4F808191810895089588E784
:1025F0008A95F1F7089500C008950C94F712089594
:102600000C94FF120C9400130C94FF120C940413FE
:10261000F894E82FE295EF70F0E031A9282F2F70A1
:1026200081E090E001C0880F2A95EAF7982F9095F5
:10263000932391AB92A9892B82AB789408950F9341
:102640001F93CF93DF93C5EFD0E089918F3F11F0B7
:102650000E94081380E0CC3FD807B9F7C7EED0E05E
:1026600005EF10E089918F3F11F00E9408130C17BD
:102670001D07C1F7DF91CF911F910F910895BF9270
:10268000CF92DF92EF92FF920F931F93CF93DF933E
:102690008C01C62FD0E0CE018B509F4F6C01FC0106
:1026A00090819F3F09F450C0B62EF894E92FE2952F
:1026B000EF70F0E081A99F7021E030E001C0220FAF
:1026C0009A95EAF7822B81AB82A92095282322AB29
:1026D00078940E94FB12E7EEF0E045EF50E021E035
:1026E00030E0E12CF12C61916F3F89F0A62FA2958B
:1026F000AF70B0E0D0968C9190E06F7002C095956D
:1027000087956A95E2F780FD02C0C90102C080E0AA
:1027100090E0E82AF92A220F331F4E175F0719F7B6
:10272000F60180818F3F11F00E94081361E0E114EF
:10273000F10409F460E08B2D0E94FD12CC0FDD1F27
:10274000C00FD11FF982E882DF91CF911F910F91C5
:10275000FF90EF90DF90CF90BF9008950E941F13DD
:102760008EE0E5E9F2E0DF01982F1D929A95E9F7F6
:10277000E7E8F2E0DF011D928A95E9F787E00E9421
:102780000E140C94C004FF920F931F93CF93DF930A
:10279000CDB7DEB72E970FB6F894DEBF0FBECDBF14
:1027A0008E010F5F1F4F8EE0F80111928A95E9F7B5
:1027B000F12C6F2DC8010E943F13F394F7E0FF1234
:1027C000F8CF4EE050E0B80187E892E00E941F2663
:1027D000FF24F394009709F4F12C892B41F08EE04B
:1027E000F801A7E8B2E001900D928A95E1F72F2D4C
:1027F00047E065E972E087E892E00E940F140E94CA
:10280000C2048F2D2E960FB6F894DEBF0FBECDBF3B
:10281000DF91CF911F910F91FF9008950895FF923E
:102820000F931F93CF93DF93F82E092F162FD72FD7
:10283000C42F222349F081E08093D4010E94142206
:102840009093D3018093D2018091D4018823D9F051
:102850008091D2019091D3010E942C22059798F08B
:10286000EF2DF02FA12FBD2F80E090E04C2F50E0F6
:102870008417950734F4219131912D933D9301965E
:10288000F7CF1092D401DF91CF911F910F91FF905C
:1028900008950E9476220E9426100C9487220E949E
:1028A00002220E946F220E9412100E9449140E946C
:1028B00095220E941C10FBCFEF92FF920F931F9363
:1028C000CF93DF938B01682F11110AC0442329F0A5
:1028D000E82FF0E0E153FC4F6491762F862F75C00E
:1028E000212F30E0E82FF0E0442321F0E153FC4FAA
:1028F000E491F0E046E0049FC0011124CFEFD0E066
:10290000BE010E9485254BEA4603C001479F900DFA
:102910001124800F911D800F911D982F990F890F01
:10292000AE01421B530B4E9FD0014F9FB00D5E9FD7
:10293000B00D11249B2F189FA0011124452F55275E
:102940008E01041B150B0E9FA0010F9F500D1E9FA3
:10295000500D11247E01E81AF108E29E8001E39EE9
:10296000100DF29E100D1124212F3327C21BD30B03
:10297000CE9F9001CF9F300DDE9F300D112462302D
:102980007105A9F048F46115710569F061307105B0
:10299000C9F48B2F752F0DC06430710581F058F08C
:1029A0006630710579F47E2F8B2F932F0DC0832F06
:1029B0007B2F9E2F09C08E2F7B2F952F05C08E2F2A
:1029C000732F02C07E2F852F692FDF91CF911F912A
:1029D0000F91FF90EF90089541E00E945C140895DC
:1029E00008950E94EC140895CF93DF93762FE901A8
:1029F000682F842F0E94F114798368838A83DF9182
:102A0000CF9108958091A302282F269530E02115BB
:102A1000310519F48170826005C02532310524F03A
:102A2000817088648093A302089588E090E00C94FC
:102A30003426CF92DF92EF92FF926B017C010E94CD
:102A40000215B701A60188E090E0FF90EF90DF90BB
:102A5000CF900C945126E3EAF2E083E08083118268
:102A60008FEF82838383148260817181828193815D
:102A70000C9419158091A30280FF02C086950895D9
:102A800080E008959091A702933018F49F5F90938F
:102A9000A702882351F06091A3027091A402809153
:102AA000A5029091A6020C941915089581E00C944A
:102AB00042159091A702992319F091509093A70283
:102AC000882351F06091A3027091A4028091A50225
:102AD0009091A6020C941915089581E00C94591553
:102AE00070E00C942B1D609168008091A30280FF20
:102AF0000AC08091670023E0829FC001112488559D
:102B00009D4F0C9470158091690090916A0089170F
:102B100080F7E82FF0E09F01220F331FE20FF31F31
:102B2000E855FD4F1182108212828F5FF0CF909195
:102B3000A30290FF16C09091690020916A0092173D
:102B400070F4E92FF0E0DF01AA0FBB1FEA0FFB1FB3
:102B5000E855FD4F8183608342839F5FF0CF0C94E3
:102B600073150895CF93DF9300D01F92CDB7DEB7D2
:102B70009091A30290FF0AC09E012F5F3F4F0E94D9
:102B8000F4144B8169818A810E9497150F900F90F0
:102B90000F90DF91CF910895CF93DF93EC01EC81FB
:102BA000F0E0E653FD4F4491E3EAF2E06281818177
:102BB0000E94B2158C818F5F8C83DF91CF91089535
:102BC000CF93DF93EC01E3EAF2E0438162818C81F1
:102BD0000E94B2158C818F5F8C83DF91CF91089515
:102BE0000F931F93CF93DF9300D01F92CDB7DEB723
:102BF0008C018091D50181110AC09E012F5F3F4F4A
:102C00004FEF6FEF0E94F4148A818093D501F80191
:102C10008481813051F028F0823061F44091D501F7
:102C20000AC08091D50140E007C06091D50140E025
:102C300080E003C040E080E060E00E949715F8016A
:102C4000848190E0019663E070E00E94992584837E
:102C50000F900F900F90DF91CF911F910F910895DA
:102C6000AF92BF92CF92DF92EF92FF920F931F939A
:102C7000CF93DF9300D01F92CDB7DEB7182FF62E7B
:102C8000042FE22E9091A30290FF6DC0E92FE695EC
:102C9000AE2FB0E0A450BF4F8C918093DF019E7F98
:102CA000923061F49E012F5F3F4F812F0E94F414F8
:102CB0004B8169818A810E94971543C0823019F443
:102CC0000091A6023EC0863019F41091A40239C0CA
:102CD0008930D9F38931A9F5E9518E2F8170D82E29
:102CE000E695F0E0E653FC4FA590B490C12CBB24D0
:102CF00060916B00C61618F52C2D30E0A29EC00125
:102D0000A39E900DB29E900D112470E00E94852527
:102D1000812FD11002C0860F01C0861B90916900DF
:102D2000290F311DA901440F551F240F351F2855A8
:102D30003D4F402F6F2D0E94F414C394D9CF0E94B1
:102D400073151093A402F092A5020093A602EE2040
:102D500051F06091A3027091A4028091A50290911C
:102D6000A6020E9419150F900F900F90DF91CF913E
:102D70001F910F91FF90EF90DF90CF90BF90AF9099
:102D80000895E3EAF2E09181282F4381628188E08F
:102D9000890F0C94301681E00C94C116E3EAF2E03E
:102DA0009181282F4381628188EF890F0C9430161E
:102DB00081E00C94CE16E3EAF2E0628121E1620F39
:102DC00008F46FEF282F438181810C94301681E045
:102DD0000C94DB16E3EAF2E0628121E1621B08F465
:102DE00060E0282F438181810C94301681E00C949F
:102DF000EA16E3EAF2E0438121E1420F08F44FEFE3
:102E0000282F628181810C94301681E00C94F91690
:102E1000E3EAF2E0438121E1421B08F440E0282F7D
:102E2000628181810C94301681E00C94081720E0B7
:102E30000C943016FF920F931F93CF93DF93EC0106
:102E4000F12C0FEF10E060916B00F616F0F480911A
:102E500069002F2D30E0280F311DC901880F991FFF
:102E6000280F391F28553D4F70E0C8010E94992551
:102E7000962F8C814091A6026091A502F99E800D4B
:102E800011240E94F414F394DECF0E9473159A81EA
:102E90008C8190FF02C08F5F01C081508C83DF91D5
:102EA000CF911F910F91FF900895AF92BF92CF9253
:102EB000DF92EF92FF920F931F93CF93DF93FC016A
:102EC000828180FF02C00FEF01C001E010E043E10A
:102ED000A42E80916B00181708F043C08091690000
:102EE000C12ED12CE601C80FD11DCE01880F991F2C
:102EF000C80FD91FC855DD4F198218821A8234E0D5
:102F0000E32EF12CB12C8091D7018B0D84312CF064
:102F10006A2D0E947725892F05C087FF03C09091F5
:102F20006B00890F082E000C990BC816D90691F476
:102F30008091A6028E9DA0018F9D500D1124559564
:102F40004795559547959E016091A5028091A402F1
:102F50000E94F414B00EF1E0EF1AF108A1F61F5F21
:102F6000B8CF0E9473158091D701013031F48111DF
:102F700002C080916B00815007C090E00196609183
:102F80006B0070E00E9499258093D701DF91CF916B
:102F90001F910F91FF90EF90DF90CF90BF90AF9077
:102FA0000895CF938091690090916A00891770F419
:102FB000E82FF0E09F01220F331FE20FF31FE855C7
:102FC000FD4F1182108212828F5FF0CFC0E06091BE
:102FD0006B00C617C0F5EC2FF0E070E0CF010E9447
:102FE000992520916900820F2091D601022E000CB4
:102FF000330B90E0E217F307CCF020916600022E2D
:10300000000C330B2E173F078CF09C01220F331F4F
:10301000820F931F9C0128553D4F4091A60260915D
:10302000A5028091A4020E94F4140BC0FC01EE0FD3
:10303000FF1F8E0F9F1FFC01E855FD4F118210826C
:103040001282CF5FC4CF0E947315209165008091DA
:10305000D601820F8093D60190916600920F9093D3
:10306000660019165CF4082E000C990B40916B0059
:1030700050E041505109841795071CF02195209389
:103080006500CF9108958F929F92AF92BF92CF9299
:10309000DF92EF92FF920F931F93CF93DF938C01F8
:1030A000FC014481C42FD0E09E01DE010E94DD2599
:1030B0009B01AC010E94F3256B017C01E0E2F0E092
:1030C000EC1BFD0BA5E5B0E09B01AC010E94F325D4
:1030D0004B015C019F01DF010E94D5259B01AC01E2
:1030E0000E94FE259B01AC012C0D3D1D4E1D5F1D58
:1030F000C501B4010E94AD25C22FD22F2A3228F477
:10310000F3E02F9F900111240DC025E530E02C1B2A
:103110003109C901880F991F280F391F37FF02C0D5
:103120002F5F3F4F35952795C22FC095F12C85E530
:10313000E82EED1A80916B00F816C8F4F1FC02C07D
:103140008E2D01C08D2F909169002F2D30E0290F19
:10315000311DA901440F551F240F351F28553D4F20
:103160004C2F6091A5020E94F414F394E3CF0E94C7
:103170007315F8018481811102C091E003C080328F
:1031800019F49FEF9093640090916400890FF80107
:103190008483DF91CF911F910F91FF90EF90DF908B
:1031A000CF90BF90AF909F908F9008950F931F93F3
:1031B000CF93DF93EC0100E010E080916B00282FAB
:1031C00030E00217130724F5909169009801290F48
:1031D000311DA901440F551F240F351F28553D4FA0
:1031E000869590E04C81081719071CF4442331F0B0
:1031F00002C0411103C04091A60201C040E06091AD
:10320000A5028091A4020E94F4140F5F1F4FD5CF36
:103210000E9473158C8190E00196817099278C83B0
:10322000DF91CF911F910F910895E3EAF2E0808141
:103230008E7F808360817181828193810E941915C4
:103240001092E0012FEB84ED91E0215080409040FE
:10325000E1F700C000000C9473156091A30266951D
:1032600070E04BE050E08CE690E00E941226892B43
:1032700019F481E08093E0010E9414229093D90117
:103280008093D80108959091A30290FF35C091706A
:10329000811102C0926006C0853210F0986402C0AD
:1032A000880F982B9093A302662351F06091A3029C
:1032B0007091A4028091A5029091A6020E94191516
:1032C0006091A302669570E04BE050E08CE690E0E0
:1032D0000E941226892B19F01092E00102C00E9470
:1032E0002D1981E08093DB014091A6026091A50237
:1032F0008091A4020C9417170895682F9091A3024F
:10330000969581E0890F853208F081E00C9443198D
:1033100081E00C947D19682F9091A30296958FEF10
:10332000890F09F484E20C94431981E00C948B1901
:1033300061E00C944319E3EAF2E0808181608083CC
:1033400086950C9498198091A30280FD0C94151910
:103350000C949B1960E00C9443198091DE0181115B
:103360002EC00E94380F811104C00E94E00F0E94FD
:103370002B150E9415156093A3027093A4028093ED
:10338000A5029093A6026E7F61F40E942B150E9405
:1033900015156093A3027093A4028093A5029093E5
:1033A000A6020E9402151092E0018091A30280FF04
:1033B00003C086950E94AA1981E08093DE010895DA
:1033C0000F931F93CF93DF938091E001882309F43B
:1033D00085C08091DF01E091A302E695E81BE093B0
:1033E000DA01823049F4F0E0EA53FD4FE491CE2F48
:1033F000D0E00CEC15E149C0863049F4F0E0ED5323
:10340000FD4FE491CE2FD0E000EE15E13EC08930B3
:1034100051F4E695F0E0E054FD4FE491CE2FD0E07A
:103420000AE117E132C08F3051F4E695F0E0E35441
:10343000FD4FE491CE2FD0E005E517E126C08531A0
:1034400049F4F0E0E654FD4FE491CE2FD0E001EDD9
:1034500017E11BC0883181F0833239F4E8EBF2E0E8
:10346000C591D49100EF15E110C0843251F4C4EF3E
:10347000D1E006ED18E109C0C8E2D0E003E418E1AC
:1034800004C0C0EDD7E000EF14E18091DB01882398
:1034900061F01092DB010E9414229093D901809375
:1034A000D8011092DD011092DC010E941422E091FB
:1034B000D801F091D9018E1B9F0B8F3F9F4770F46D
:1034C000EC0FFD1FF093D901E093D80188ED91E056
:1034D000F801DF91CF911F910F910994DF91CF9166
:1034E0001F910F910895882311F0FA0101C0FB018B
:1034F0000994CF93DF93C82FD62F0E943A158C17CB
:1035000040F00E943A158D1720F4DF91CF910C9472
:1035100088198C2FDF91CF910C9498191F93CF931A
:10352000DF93FB0112811111C3C0EC010E94550E03
:103530008272CD3CFCE5DF0709F49AC0A8F5C73CD0
:10354000ECE5DE0709F476C0A8F4C43C9CE5D90795
:1035500009F45FC028F4C33CDC4509F457C054C0EB
:10356000C53C9CE5D90709F459C0C63CDC4509F4C3
:103570005CC04AC0CA3CFCE5DF0709F46AC050F4ED
:10358000C83CECE5DE0709F45AC0C93CDC4509F447
:103590005BC03AC0CB3C9CE5D90709F45FC0CC3C8A
:1035A000DC4509F460C030C0C23DFCE5DF0709F42A
:1035B0006FC088F4CF3C9CE5D90709F460C008F4DB
:1035C0005CC0C03DFCE5DF0709F45CC0C13DDC45E3
:1035D00009F45BC019C0C53D9CE5D90709F460C07A
:1035E00050F4C33DFCE5DF0709F455C0C43DDC459C
:1035F00009F454C009C0C63D9CE5D90709F455C07B
:10360000CE35DD4509F454C011E052C00E94A31923
:103610004FC045E959E168E879E104C048E859E15B
:1036200065E979E10E94731A43C048ED56E16BECFD
:1036300076E1F8CF4BEC56E168ED76E1F3CF46EF5B
:1036400056E167EE76E1EECF47EE56E166EF76E1C2
:10365000E9CF44E157E165E077E1E4CF45E057E1A8
:1036600064E177E1DFCF4DE655E166E575E1DACF5C
:1036700046E555E16DE675E1D5CF81E017C065E01F
:1036800082E010C068E086E00DC06EE089E00AC00C
:1036900064E18FE007C067E185E104C088E106C00E
:1036A00062E289E10E94791A03C083E20E949819BC
:1036B000812FDF91CF911F91089586E090E00C94C7
:1036C0002C26682F86E090E00C9440268091E10241
:1036D000847089618093E1020C94611B0E94380F11
:1036E000811104C00E94E00F0E94661B0E945D1BB6
:1036F0008093E102282F26952695269530E02430E8
:10370000310524F0877088618093E1028091E102A5
:1037100080FF04C086958695869501C080E00C9454
:103720007F1C2091E102822F869586958695482FF1
:1037300050E04330510554F48F5F982F990F990F43
:10374000990F822F8770892B8093E1028091E1028B
:1037500081608093E1020E94611B8091E102869565
:10376000869586950C947F1C8091E102982F969502
:1037700096959695A1F0915E990F990F990F877084
:10378000892B8093E102887F91E009F490E0809199
:10379000E10290FB80F98093E1020E94611B80911D
:1037A000E1028695869586950C947F1C8091E102B6
:1037B00080FD13C081608093E102813019F489E0BB
:1037C0008093E1028091E1020E94611B8091E102FD
:1037D0008695869586950C947F1C08958091E102CC
:1037E00080FF08C08E7F8093E1020E94611B80E011
:1037F0000C947F1C08958091E10280FD0C94EE1BD7
:103800000C94D61B9091E102892F8695869586951A
:103810008F5F8F719770843038F4880F880F880F0E
:10382000892B8093E10202C09093E1028091E10232
:10383000887F91E009F490E08091E10290FB80F9AB
:103840008093E1020E94611B8091E102869586953A
:1038500086950C947F1C843008F083E09091E102FF
:103860009770282F220F220F220F922B9093E102A4
:10387000987F21E009F420E09091E10220FB90F98B
:103880009093E1020C947F1C0E942B1C8091E1021A
:103890000C94611B9C01FB018281882349F12E3B22
:1038A000FCE53F07C9F040F42C3BECE53E0769F02E
:1038B0002D3B3C4561F00895203C9CE5390791F093
:1038C00070F0213C3C4589F0089583E001C080E020
:1038D0000E94441C80E008950E94B41BFBCF0E940C
:1038E000911BF8CF0E94FB1BF5CF0E94021CF2CF68
:1038F00081E008958C9A94980895949808958F92F1
:103900009F92AF92BF92CF92DF92EF92FF920F936E
:103910001F93CF93DF93C82F843040F4811107C0E9
:103920008FB58F7D8FBD0E947D1C04C0C3E08FB515
:1039300080628FBDA6B5B7B52C2F30E00E94DD2583
:1039400023E030E040E050E00E94AD250027122F38
:10395000232F342F012F122F232F332786B597B50E
:103960006CE070E00E9485256017710730F0C80197
:1039700069E070E00E94852552C086B597B5E6B42F
:10398000F7B4E6B5F7B5C6E0D0E0BE010E948525E4
:10399000060F171F211D311D4801590185E0880CB4
:1039A000991CAA1CBB1C8A95D1F7C701BE010E94B5
:1039B00085256F01E12CF12CA7019601260F371FF9
:1039C000411D511DC501B4010E94AD2569017A0157
:1039D000E6B5F7B5CA01B9010E9467259B01AC01A4
:1039E000DF010E94F3259B01AC01C701B6010E94D3
:1039F0006725DC01CB012FE0B695A79597958795B4
:103A00002A95D1F706B517B520E030E00817190759
:103A10002A073B0718F466B577B5CB01BC0179BD21
:103A200068BDDF91CF911F910F91FF90EF90DF90D4
:103A3000CF90BF90AF909F908F90089508950E946F
:103A40007A1C82E28FBD89E18EBD8FEF9FEF97BD1B
:103A500086BD0C946E1B0F931F93CF93DF938C0145
:103A6000EB018091E101811105C00E946F2081E08E
:103A70008093E101AE01440F551F4C0F5D1F24E6FA
:103A800030E0B80180EBDF91CF911F910F910C9442
:103A90002221CF93DF93EC01FB018281882309F47B
:103AA0003CC1C430FDE5DF0760F4CB3F9CE5D9079E
:103AB00088F49E0122503C452431310508F02EC186
:103AC00009C0C236EDE5DE0729F0C63AFDE5DF079D
:103AD00009F024C10E944B0F9093860280938502C7
:103AE000C1318CE5D80709F4C6C008F042C0C9301E
:103AF000ECE5DE0709F49BC000F5C5308CE5D8077E
:103B000009F485C078F4C330ECE5DE0709F478C029
:103B100008F07AC0C230DC4509F0F5C0809185021A
:103B20008160EFC0C7309CE5D90709F478C008F080
:103B30007AC0809185028061E4C0CD30FCE5DF076A
:103B400009F487C058F4CB309CE5D90709F479C053
:103B500008F07BC08091850288606FC0CF30FCE5A3
:103B6000DF0709F480C008F082C080918502877F5A
:103B7000C8C0CE3F9CE5D90709F471C000F5C53136
:103B8000FCE5DF0709F485C068F4C3319CE5D9077B
:103B900009F475C008F095C00E9402098091850261
:103BA0008F77AFC0CC3FFCE5DF07A9F108F054C028
:103BB000CB3FDC4509F0A7C08091860240C0C230EF
:103BC000EDE5DE0709F489C058F4C1158DE5D80785
:103BD00009F45AC008F069C08091860282602FC043
:103BE000C236EDE5DE0709F47CC0C63AFDE5DF0725
:103BF00009F481C0C330DD4509F085C080E06EC0A6
:103C00008091850282607DC08091850216C080917E
:103C10008502886076C08091860282604FC0809164
:103C2000850280626EC08091850280646AC00E94B5
:103C3000020980918502806864C0846062C08160EE
:103C40003DC0809185028E7F5CC0809185028D7F12
:103C500058C08091850216C08091860218C080915C
:103C600086028D7F2BC0809185028F7E4AC0809115
:103C700085028F7D46C0809185028F7B42C08091F6
:103C80008502877F8B7F3DC0809186028D7F8E7FEE
:103C900015C08091850282FB222720F991E09227AE
:103CA00090FB82F990FB83F92CC080918602982FBB
:103CB000909591708E7F892B90FB81F9809386027D
:103CC00022C00E9402098091850287FB222720F9E9
:103CD00091E0922790FB87F914C081E00E94E20FE7
:103CE00012C08091850284FB222720F991E092275F
:103CF00090FB84F906C080918502982F909590FBE7
:103D000080F98093850280918502909186020E94BD
:103D10005C0F0E94020980E001C081E0DF91CF9139
:103D200008950F931F9341E050E060E070E08A0136
:103D30009B0104C0000F111F221F331F8A95D2F769
:103D4000C901B8010E945A091F910F910C940209F0
:103D50008B3109F468C058F58B3009F486C078F4CB
:103D6000863009F445C020F4853009F44BC07FC08B
:103D7000873009F44AC0883009F477C078C08031B0
:103D800009F464C068F48E3009F071C08091D101EB
:103D900082FB222720F991E0922790FB82F94CC008
:103DA000863109F462C0893109F45FC060C08A328B
:103DB000E1F060F4873209F455C028F48E3108F43C
:103DC00056C08D5150C08932E9F051C0833450F44F
:103DD0008A3308F045C0853309F444C0883309F4B8
:103DE00044C045C08334F1F142C00E94E00F3DC0A1
:103DF0008091D101817F8E7F8093D10181E080937A
:103E0000E20108950E94C50430C08091D101982F2D
:103E10009095917090FB80F98093D101911125C00C
:103E2000897F877F10C08091D10181FB222720F9F3
:103E300091E0922790FB81F98093D1019923A9F019
:103E40008091D10181608093D1010FC08091D10117
:103E500083FB222720F991E0922790FB83F9ECCF96
:103E6000895301C080E00E94911E81E0089580E0A6
:103E7000089580E008950C94391FCF93C82F809146
:103E8000E201882319F0813031F02BC00E94550ED9
:103E9000823249F504C00E94550E823261F48C2FA3
:103EA0000E943B1F811104C08C2F0E94A81E17C0C6
:103EB00081E090E014C08C2F0E94391F81110EC048
:103EC000C43149F018F4CB3049F00FC0C93219F0B1
:103ED000C83321F00AC01092E20107C081E081706E
:103EE00006C01092E20180E002C080E0F8CFCF91DE
:103EF0000895CF93DF9386319C4541F5EB010E94F5
:103F0000550E982F8A81209162003091630088239A
:103F100079F09A7A81E009F480E08093E3019111CD
:103F200002C069E201C065E3C9010E94D7210AC04D
:103F30008091E301811102C069E201C065E3C9011A
:103F40000E94D9210E94970E80E001C081E0DF919C
:103F5000CF9108950F931F93CF93DF93C42FD22F48
:103F6000FC0182818823C9F04093E6010E9414225B
:103F70009093E5018093E40180E28C0F883008F093
:103F800057C0C77081E001C0880FCA95EAF7DF917A
:103F9000CF911F910F910C946E068091E60148130A
:103FA00030C08091E4019091E5010E942C22883C70
:103FB000910538F510E21D0FCD17B9F080E28C0F96
:103FC000883040F4C77081E001C0880FCA95EAF7D5
:103FD0000E947506183028F581E09D2F977001C06A
:103FE000880F9A95EAF70E946E06802F0E94650658
:103FF0001830F0F4D77081E001C0880FDA95EAF745
:104000000AC080E28C0F883098F4C77081E001C04C
:10401000880FCA95EAF7DF91CF911F910F910C9409
:104020007506802FDF91CF911F910F910C9465063B
:10403000DF91CF911F910F9108950F939C01CB01B8
:10404000243F4CE5340731F188F4293DFCE53F0776
:10405000D9F02A3D4CE5340779F1283D3C45A9F5D6
:1040600006E221EE41EE68ED7CE52BC0263FFCE543
:104070003F07E1F0A8F0273F3C4539F507E225EE80
:1040800046EE67EF7CE51DC007E225EE45EE69EDE3
:104090007CE517C006E221EE40EE64EF7CE511C03E
:1040A00007E225EE44EE65EF7CE50BC006E221EE6B
:1040B00042EE66EF7CE505C008E221E045EE6AEDE0
:1040C0007CE50E94AA1F80E008C0FC018281882351
:1040D00019F01092E60101C081E00F91089511B826
:1040E00087E080B985B3836085BB86B7846086BF6F
:1040F00086B7816086BF86B7806486BF08959F9229
:10410000AF92BF92CF92DF92EF92FF920F931F93E5
:10411000CF93DF93B82EEB010E9414226C01C431BF
:10412000D10558F0CF3F8FEFD80759F0CE0164E1A9
:1041300070E00E9485257B0107C0EE24E394F12CFA
:1041400003C025E0E22EF12C84E8A82E94EA992EF3
:1041500016BE96BE0E9414228C0106B607FC08C04B
:104160000E941422801B910B8E159F05B0F324C072
:1041700081B1887F883039F081B1887F803119F032
:104180000FEF1FEF1BC0B3B8A6BE0E9414228C0114
:1041900006B607FC08C00E941422801B910B8E15E6
:1041A0009F05B0F309C081B1887F883111F0803458
:1041B00039F700E010E00DC00EEF1FEFCF3F8FEF9B
:1041C000D80731F2C6010E942C228C179D0708F4F3
:1041D000BFCFC801DF91CF911F910F91FF90EF905A
:1041E000DF90CF90BF90AF909F9008950F931F9353
:1041F000CF93DF93EB0183B984E886BF0E9414223A
:104200008C0106B607FC0EC0CF3F8FEFD807C9F36D
:104210000E941422801B910B8C179D0790F38EEF48
:104220009FEF0BC021B1287F81E090E0283211F48C
:1042300080E090E0919581959109DF91CF911F9158
:104240000F910895CF92DF92EF92FF920F931F93F9
:10425000CF93DF936B018A017901B9010E947F201E
:10426000E6010C0D1D1DC017D10759F424E926BF26
:10427000DF91CF911F910F91FF90EF90DF90CF9042
:10428000089597FDF3CFB70189910E94F620EBCFF7
:10429000909323018093220108959093EC018093E1
:1042A000EB010895E091EB01F091EC01309721F0E2
:1042B0000190F081E02D099480E00895E091EB01F8
:1042C000F091EC01309721F00280F381E02D099408
:1042D00008952091E9013091EA012817390771F01A
:1042E0009093EA018093E901E091EB01F091EC01F8
:1042F000309721F00680F781E02D099408952091F0
:10430000E7013091E8012817390771F09093E8012F
:104310008093E701E091EB01F091EC01309721F0FF
:104320000084F185E02D09940895FC01329697E010
:1043300080E0915029F021912223D9F38F5FF9CFAA
:104340000895662349F0FC01329608962191621780
:1043500029F0E817F907D1F780E0089581E0089582
:104360009C01FC0132969FEF80E04191461789F055
:104370009F3F19F4411101C0982F8F5F8630A9F734
:104380009F3F39F0F901E90FF11D97FDFA9562831E
:10439000089508959C012A5F3F4FFC014281461316
:1043A00001C01282019682179307B9F708950C9401
:1043B000B0210C94CA21029626E0FC0111922A95A4
:1043C000E9F7089508950C94E2210C94E3210C94EC
:1043D000E2210C94E2210C94E221CF930E94E92186
:1043E0000E94C3130E94E721C0E08C2F0E94ED12AF
:1043F000892B29F4CF5FC730C1F780E001C081E08D
:10440000CF91089508958091EF0181110C943405A6
:1044100008950E9402090C943B058BE083BF8BEB4F
:104420008CBF82E089BF08952FB7F8948091E20293
:104430009091E302A091E402B091E5022FBF0895AC
:104440002FB7F8946091E2027091E3028091E40248
:104450009091E5022FBF08959C014FB7F894809189
:10446000E2029091E302A091E402B091E5024FBF15
:10447000821B930B089578941F920F920FB60F92A0
:1044800011248F939F93AF93BF938091E2029091F9
:10449000E302A091E402B091E5020196A11DB11DD5
:1044A0008093E2029093E302A093E402B093E502CA
:1044B000BF91AF919F918F910F900FBE0F901F9062
:1044C000189560E081E090E00E9463269CE088E11E
:1044D0000FB6F894A89581BD0FBE91BDFFCF0E9485
:1044E00014229093EE018093ED0108950E944C25D3
:1044F0008B9A80E0815041F0A895E7EBFBE0319783
:10450000F1F700C00000F6CF8B98789408950E94D0
:1045100074230E944D212FEB84ED91E021508040C7
:104520009040E1F700C00000089580910D038823BA
:1045300089F010920D030E9414229093EE01809353
:10454000ED018091EF018823D1F11092EF010E94DB
:10455000092211C08091EF01811111C08091ED01FC
:104560009091EE010E942C22069728F081E0809322
:10457000EF010E9403228091EF01882301F10E9444
:1045800003220E94ED21882339F1F89421B3939AF4
:10459000822F8C6081BB92B38CE0982792BB3FE561
:1045A0004AEE90E0315040409040E1F700C00000FA
:1045B00092B3892782BB21BB9398789408950E9477
:1045C000552480911303882329F08091F10284FD02
:1045D0000E94CD100C941B230895809184020895AD
:1045E00008959091F501981307C02091F30130913F
:1045F000F40126173707A9F08093F5017093F401B1
:104600006093F3018093F0017093F2016093F101E4
:1046100080912A0384FF05C063E080EF91E00C9451
:1046200051240895BC0184E00C94F122BC0183E084
:104630000C94F1220895CF93DF93CAE0D0E08091EB
:10464000F10284FF18C08091010290910202981734
:10465000E1F028E0829FC001112468E08D5F9D4F4A
:104660000E944D248091010290E001968F7099275D
:10467000809301020AC00E94552487EB9BE00197BA
:10468000F1F700C000002197D1F6DF91CF91089596
:10469000CF93DF93EC01A0910202B0E0CD0101962F
:1046A0008F70992720910102281779F093E0AA0FC3
:1046B000BB1F9A95E1F7AD5FBD4F98E0FE010190F9
:1046C0000D929A95E1F7809302020E9455240E9470
:1046D0001B2388E0FE01A9EFB1E001900D928A95BD
:1046E000E1F7DF91CF91089587E790E00895FC010D
:1046F000808180768032A1F58181813061F484816E
:104700009581892B69F589EF91E090930F03809350
:104710000E0388E00895823041F483E892E090939C
:104720000F0380930E0381E008958A3021F4838182
:104730008093830215C0893099F482819381811519
:10474000924081F484819581892B61F481E080938A
:10475000F801868197819093F7018093F60102C05A
:1047600080E008958FEF08952091F6013091F701D0
:10477000232B71F02091F801213051F4FC0180814C
:10478000809384021092F7011092F60181E008955F
:104790008FEF08950895FC0193819330B1F068F490
:1047A000913081F0923009F054C08FEC94E09093F6
:1047B0000F0380930E038BE30895913221F192321F
:1047C00091F147C08AE095E018C08281813099F06C
:1047D00050F08230F1F58CE195E090930F038093D7
:1047E0000E0380E1089582E495E090930F03809397
:1047F0000E0384E008958EE295E090930F0380937A
:104800000E0382E108958281882329F0813009F521
:104810008AEF94E002C081EE94E090930F038093BE
:104820000E0389E0089584819581009751F00197E6
:1048300081F486E495E090930F0380930E0382E366
:10484000089588E795E090930F0380930E0380E42A
:10485000089580E008951F93CF93DF93162FEA0108
:10486000288124FF05C0398128E82327298302C035
:104870002AE52883212FFC01CE010296DC0131912B
:104880003D9321501216DCF3612F0E9410031C5F30
:104890001883DF91CF911F91089541EF52E00C945E
:1048A0002B244AE253E00C942B24CF93DF936091A6
:1048B0001003635067FD93C080910C03CCE0D0E0FF
:1048C000C81BD109CC5EDC4F80910B03803120F4F2
:1048D000CE010E94CA2381C08D3209F06EC06830BB
:1048E00009F07BC083EC8093E6028AE58093840024
:1048F00010920A038881807621F0CE010E947723EE
:1049000049C09A811092EF028981811106C01092EC
:10491000F0022FEE32E082E038C0853019F4909337
:10492000110330C08630A1F48B81813041F0823098
:1049300031F0833021F0813211F0823221F4CE0146
:104940000E94CB2301C080E090E490930A0322C030
:10495000883089F0893019F49093130313C08A309A
:1049600069F08B3079F48BE48093F20280932B030F
:104970008093FE0207C023E133E002C02FEE32E055
:1049800081E003C02FEE32E080E030930F032093EC
:104990000E0309C08F3F39F4988197FD8E8190E80E
:1049A00090930A0307C09F81911104C09E819817BC
:1049B00008F4892F8093830010C080910A0387FF39
:1049C0000CC0CE010E94B4238F3F21F48EE180936E
:1049D000840003C081111092830010921003809113
:1049E000840084FF4CC0809183008F3F09F447C04E
:1049F000C82F893008F0C8E08C1B80938300909109
:104A0000E60288E889278093E602CC2359F1809159
:104A10000E0390910F0320910A0326FF12C0A6EE09
:104A2000B2E02C2FAC01465E5240FA01EA0FFB1FA8
:104A3000E4911196EC931197215011962111F5CF25
:104A400008C0E7EEF2E0DC012C2F3D9131932150BC
:104A5000E1F701962FEF2C0F820F911D90930F031A
:104A600080930E036C2F87EE92E00E941003CC5FC0
:104A7000CC3019F08FEF80938300C093840084E1E1
:104A800090B39C7031F48150D9F7109211031092B9
:104A90000903DF91CF910895CF93DF9385B78860A5
:104AA00085BF8BB780688BBFC1EFD2E08BE4898371
:104AB000AAE2B3E011968C931197EDEFF2E08183B7
:104AC0008AE588838C938083DF91CF910895DB0101
:104AD0008F939F930E94F325BF91AF91A29F800D6A
:104AE000911DA39F900DB29F900D1124089587FBF7
:104AF000082E062687FD819567FD61950E94062692
:104B00000EF4919507FC81950895AA1BBB1B51E1FA
:104B100007C0AA1FBB1FA617B70710F0A61BB70B2D
:104B2000881F991F5A95A9F780959095BC01CD01D2
:104B3000089597FB072E16F4009407D077FD09D04F
:104B40000E94852507FC05D03EF4909581959F4FE6
:104B50000895709561957F4F0895A1E21A2EAA1BC2
:104B6000BB1BFD010DC0AA1FBB1FEE1FFF1FA2171D
:104B7000B307E407F50720F0A21BB30BE40BF50B1A
:104B8000661F771F881F991F1A9469F760957095A3
:104B9000809590959B01AC01BD01CF010895EE0F6A
:104BA000FF1F0590F491E02D09940E94DD25332329
:104BB00012F48A1B9B0B0C94EE25A29FB001B39FAD
:104BC000C001A39F700D811D1124911DB29F700D16
:104BD000811D1124911D08950E94DD25B7FF0895C0
:104BE000821B930B08950E94DD25A59F900DB49F15
:104BF000900DA49F800D911D11240895B7FF0C9472
:104C0000F3250E94F325821B930B0895991B79E0ED
:104C100004C0991F961708F0961B881F7A95C9F74C
:104C200080950895FC014150504030F001900616E7
:104C3000D1F73197CF010895882799270895FB016F
:104C4000DC0104C08D910190801921F44150504045
:104C5000C8F7881B990B0895E199FECF9FBB8EBBC7
:104C6000E09A99278DB30895A6E1B0E044E050E0C2
:104C70000C947226A8E1B0E042E050E00C94722659
:104C8000262FE199FECF9FBB8EBBE09A01970DB214
:104C9000021631F02DBB0FB6F894E29AE19A0FBEDE
:104CA00008950396272F0E9441260E944026252F13
:104CB0000E944126242F0C9441260196272F0E9402
:104CC00041260C944026262FE199FECF9FBB8EBB38
:104CD0002DBB0FB6F894E29AE19A0FBE01960895A3
:104CE000DC01CB01FC01E199FECF06C0FFBBEEBBAE
:104CF000E09A31960DB20D9241505040B8F70895A8
:044D0000F894FFCF55
:104D0400C800B101010102001300131301191A1B99
:104D14001C1D1E1F202122ED2248231A23162312B4
:104D240023F022FF5AE200E900EA00B500B600B71A
:104D340000CD008301CC008A019201940121022359
:104D44000224022502260227022A02B300B4006FBD
:104D5400007000818283E200E900EA00B500B60039
:104D6400B700CD008301CC008A0192019401210295
:104D7400230224022502260227022A02B300B400D9
:104D84006F0070008182830732333435363797964B
:104D94009594939190606162636465660001020278
:104DA40002020606060909090909090F0F0F0F0F68
:104DB4000F1515151819191919191919191919236C
:024DC4002400C9
:00000001FF
